:020000040000FA
:06000000703002303A28C6
:08000800A000030EA100831209
:100010008B1C32288B1031181428B11C3228643004
:10002000010203183128182800001628172818285C
:1000300019281A281B281C281D281E281F283110A3
:10004000B114A810031005190314AA0DA90DA80DC9
:10005000B00B322831152A08AF002908AE00280855
:10006000AD00B11081010B11210E8300A00E200EF6
:02007000090085
:0C007400203084008001840A80300402E7
:10008000031C3C281230B0005E2183160C3085051D
:1000900087018312850187010730990000309A009B
:1000A000103083168E008312603083168F00831207
:1000B0000030831691009F008312C83083168100A0
:1000C000831231309000003083168C008312103080
:1000D0008B00AC2181018E018F010B118B100B1055
:1000E0008C018B178220311998204021B30B802876
:1000F000031085190314B90DF03039020319E920F2
:10010000AF2172286400311808000B1D08000B1184
:10011000B11031141230B000051D9328321483162B
:10012000011383120800321083160117831208008E
:1001300031110130B7008B132030370783169B0035
:100140001C141A088312A400A500C030A5061030A4
:10015000370783169B001C141A088312A300003073
:10016000370783169B001C141A088312A2008B17F2
:10017000321CC02822090339A200A309A409A50939
:1001800022082D02031DE32823082E02031DE32865
:1001900024082F02031DD52801303702031DD5285E
:1001A0003D18D5283D143E14852125082F02031D36
:1001B000E32801303702031DE2283D1CE2283D10F0
:1001C0003E14A921E328B70A0230370203180800B9
:1001D0009B280130B600B300B400B500B70085011C
:1001E0008701B1138220B30B0F2903108519031463
:1001F000B90DF030390203193629B41F8501B41F37
:100200008701B40B0F293708B6080319B600031984
:100210000D29FF3085008700B6039630B400311DEC
:10022000F2283111321C19292D090339AD00AE090C
:10023000AF092F1CB1132F1CF228B11BF2282E1866
:10024000F228B1178B1320303707BB002F08BA00F4
:10025000492110303707BB002E08BA004921003071
:100260003707BB002D08BA0049218B17850187018C
:10027000B70AB60102303702031CF228AC2108008D
:100280003E1C08003E101030BB003D08BA0049215A
:1002900008008B133A0883161C159A0083123B083A
:1002A00083169B0055309D00AA309D009C1464006D
:1002B0009C1857291C1183128B17080083161030C5
:1002C0009B001C141A088312BD00831620309B006B
:1002D0001C141A088312DF00831670309B001C1454
:1002E0001A088312D6000E07D7005707D800560702
:1002F000DB005807DA005607D9005807D5007030E0
:10030000BB005708BA00492108000130BD00043085
:10031000C200C5000530C400C600CA000730C100D5
:10032000C300C700C800C9005F19C1175F19C21711
:100330005F19C317DF19C4175F1AC5175F1AC617ED
:100340005F1AC7175F1AC8175F1BC917DF18CA17CC
:1003500008008501870108003D188521080001304B
:100360003D05031908005F19B7295C1805165F19C8
:10037000BB29DC1885165F19BF295C190514DF1924
:10038000C329DC1985145F1AC7295C1A87145F1A00
:10039000CB29DC1A07155F1ACF295C1B07145F1ADB
:1003A000D329DC1B87165F1BD7295D180716DF18BA
:1003B000DB29DD188715E6300E02031CF3295F1DCB
:1003C00005165F1D85165F1D0514DF1D85145F1E54
:1003D00087145F1E07155F1E07145F1E87165F1FB9
:1003E0000716DF1C87158F08031908008F01850188
:1003F00087015508DE00F123D5005608DE00F12301
:10040000D6005708DE00551CF123D7005808DE003F
:10041000D51CF123D8005908DE00551DF123D90061
:100420005A08DE00D51DF123DA005B08DE00551EF8
:10043000F123DB005F1D362AC11B312AC11C0512C6
:10044000C11C252A051258190516CB0B472A560838
:10045000CB00C101D51BC114D81BC1105818C11045
:10046000472A0512CB0B472AC103472AC1080319A3
:1004700005160319472ACB0B472AD51BC10355087C
:10048000CB00D5185C14D51E5C10D51D5C105F1D0B
:10049000632AC21B5E2AC21C8512C21C522A851204
:1004A00058188516CC0B742A5608CC00C201D61BEE
:1004B000C2145A18C210D619C210742A8512CC0B55
:1004C000742AC203742AC208031985160319742AF0
:1004D000CC0B742AD61BC2035608CC00D61ADC14E7
:1004E000561DDC10561FDC105F1D902AC31B8B2A83
:1004F000C31C0510C31C7F2A05105A190514CD0B07
:10050000A12A5708CD00C301D71BC314D51AC310A5
:10051000D719C310A12A0510CD0BA12AC303A12A04
:10052000C308031905140319A12ACD0BA12AD71B4F
:10053000C3035708CD00571A5C15571F5C11D71D10
:100540005C11DF1DBD2AC41BB82AC41C8510C41C45
:10055000AC2A8510D51B8514CE0BD92A5808CE009D
:10056000C401D81BC414D71AC410D819C410D92A6E
:100570008510CE0BD92AC403D92ADF1FC82ACE0B77
:10058000D92A5808CE00D51BDC15DA1FDC11D92A70
:10059000C408031985140319D92ACE0BD92AD81BEC
:1005A000C4035808CE00581ADC15D81FDC11D81D1A
:1005B000DC115F1EF52AC51BF02AC51C8710C51C5F
:1005C000E42A8710D51A8714CF0B062B5908CF00C1
:1005D000C501D91BC514561AC510D81BC510062B4A
:1005E0008710CF0B062BC503062BC50803198714EC
:1005F0000319062BCF0B062BD91BC5035908CF00B7
:10060000D91B5C16D91F5C12D91C5C125F1E222BF1
:10061000C61B1D2BC61C0711C61C112B0711D71A90
:100620000715D00B332B5A08D000C601DA1BC614AD
:10063000D51AC610D619C610332B0711D00B332B81
:10064000C603332BC608031907150319332BD00B28
:10065000332BDA1BC6035A08D0005A1ADC165A1E6E
:10066000DC12DA1FDC125F1E4F2BC71B4A2BC71C84
:100670000710C71C3E2B071059190714D10B602B0C
:100680005B08D100C701DB1BC714D719C710DB19E2
:10069000C710602B0710D10B602BC703602BC70856
:1006A000031907140319602BD10B602BDB1BC70345
:1006B0005B08D100DB195C17DB1D5C135B1E5C1350
:1006C0005F1E7C2BC81B772BC81C8712C81C6B2B8A
:1006D000871258198716D20B8D2B5608D200C801E5
:1006E000D91BC8145A19C810551AC8108D2B871257
:1006F000D20B8D2BC8038D2BC8080319871603193D
:100700008D2BD20B8D2BD71BC8035908D200561A3C
:10071000DC17561EDC13DA1FDC135F1FA92BC91B65
:10072000A42BC91C0712C91C982B071255190716B0
:10073000D30BC32B5808D300C901D61BC914D91A2F
:10074000C910D819C910C32B0712D30BC32BC90367
:10075000C32B5F1CB42BD30BC32B5708D300D61B62
:100760005D14D81F5D10C32BC908031907160319A0
:10077000C32BD30BC32BD51AC9035808D300D61BE0
:100780005D14D81F5D10DF1CDF2BCA1BDA2BCA1CBF
:100790008711CA1CCE2B8711D51B8715D40B0800D7
:1007A0005508D400CA01D51BCA14561ACA10D61946
:1007B000CA1008008711D40B0800CA030800CA0831
:1007C0000319871503190800D40B0800D81BCA03A6
:1007D0005608D400591ADD14591EDD10DA1FDD1039
:1007E0000800C001DE080319DE035E184014DE1A9B
:1007F00040144008C0015E1C4014DE1E4014C005B9
:06080000C00C5E0C0800B4
:084000000D000300060005009D
:02400E00CC33B1
:10420000010003000300030003000200020002009B
:1042100002000000000000000000FF00FF00FF009F
:10422000000000000000000000000000000000008E
:104230000000C000C000C000C000FF00FF00FF0081
:104240000300C300F300CF00FF00C300F300CF0062
:10425000FF00C300F300CF00FF00FF00FF00FF00DE
:10426000FF00FF00FF00FF00FF00FF00FF00FF0056
:10427000FF00FF00FF00FF00FF00FF00FF00FF0046
:10428000FF00FF00FF00FF00FF00FF00FF00FF0036
:10429000FF00FF00FF00FF00FF00FF00FF00FF0026
:1042A000FF00FF00FF00FF00FF00FF00FF00FF0016
:1042B000FF00FF00FF00FF00FF00FF00FF00FF0006
:1042C000FF00FF00FF00FF00FF00FF00FF00FF00F6
:1042D000FF00FF00FF00FF00FF00FF00FF00FF00E6
:1042E0000200BA00FF00FF00FF00FF00FF00FF0018
:1042F000FF00FF00FF00FF00FF00FF00FF00AA001B
:00000001FF
